:100000000C945D000C94CC010C947A000C947A0052
:100010000C947A000C947A000C947A000C947A0078
:100020000C947A000C947A000C947A000C947A0068
:100030000C947A000C947A000C947A000C947A0058
:100040000C947A000C947A000C947A000C947A0048
:100050000C947A000C947A000C947A000C947A0038
:100060000C947A000C947A00040309041C037700B2
:10007000770077002E006600690073006300680057
:100080006C002E00640065000E0355005300420012
:1000900061007300700012011001FF000008C0161B
:1000A000DC050401010200010902120001010080C7
:1000B0001909040000000000000011241FBECFEF4A
:1000C000D4E0DEBFCDBF11E0A0E0B1E0EAEEF2E1A6
:1000D00002C005900D92A230B107D9F711E0A2E05D
:1000E000B1E001C01D92AA34B107E1F70E94E90511
:1000F0000C9473090C94000085B7836085BF8BB79F
:1001000080648BBF08951F93CF93DF936091280184
:10011000635067FD13C080912501CCE0D0E0C81B7F
:10012000D109C45DDE4F809124018D3209F462C093
:100130008091020187FD84C0109228018091000106
:1001400084FF4AC0609101016F3F09F445C06930E6
:1001500070F16850609301018091180198E8892737
:100160008093180168E08091020187FD8BC0209187
:1001700026013091270186FF6DC0A9E1B1E080E042
:1001800090E0F901E80FF91FE491ED9301966817EB
:10019000C1F76150862F90E06F5F0196820F931F29
:1001A0009093270180932601162F1C5F0BC010929D
:1001B00001018091180198E889278093180166232E
:1001C00091F614E089E191E0E3D01C3019F08FEF53
:1001D000809301011093000194E186B3837031F4A0
:1001E0009150D9F71092290110922301DF91CF91FC
:1001F0001F910895683009F09FCF83EC8093180118
:100200008AE580930001109202018881807659F579
:100210009A81109221018981882309F043C01092AC
:10022000220122E081E291E0909327018093260150
:100230008F81882319F49E81921708F1922F1FC095
:10024000CE01D9D48F3F51F1882309F475CF109294
:10025000010172CF962FD901E9E1F1E08D918193EF
:100260009150E1F796CFCE0119D6282F8F3F01F795
:10027000888187FD25C09FEF80E8809302019093DD
:1002800001015ACF89E191E092D5682F893008F4B5
:1002900053C08FEF809301011EE19CCF8EE18093CC
:1002A00000014ACF853071F0863091F0883031F10D
:1002B000893061F18A3031F120E081E291E0B4CF00
:1002C0009E81DACF9093290120E081E291E0ACCFCA
:1002D0008B81813049F18230F9F0833029F020E0C0
:1002E00080E480930201A4CF992349F588E690E049
:1002F000909327018093260124E0F2CF21E08BE246
:1003000091E092CF21E081E291E08ECF90932B019A
:1003100020E081E291E088CF88EA90E09093270185
:100320008093260122E1DCCF86E990E090932701BB
:100330008093260122E1D4CF182F1C5F43CF913048
:1003400051F0923061F688E890E090932701809315
:1003500026012EE0C5CF8CE690E090932701809394
:1003600026012CE1BDCFA82FB92F80E090E041E01D
:1003700050EA609530E009C02D91822797958795C6
:1003800010F084279527305EC8F36F5FA8F30895B7
:10039000EADF8D939D930895CF93CFB7CF93C39505
:1003A000B09BE9F7B09B09C0B09B07C0B09B05C0EC
:1003B000B09B03C0B09B01C0A1C0DF93C0912501D9
:1003C000DD27C45DDE4FB09B02C0DF91EBCF2F93E2
:1003D0000F931F9306B32FEF00FB20F94F933F932A
:1003E00016B34FEF012700FB21F93BE031C04E7FF0
:1003F000012F16B3216028C0102F4D7F226000000E
:1004000006B329C04B7F2460012F000016B32BC018
:1004100016B3477F28602AC04F7E06B320612CC0E8
:100420004F7D16B320622FC04F7B06B3206432C0CD
:10043000422706B349934FEF0000102710FB20F925
:1004400016B31370C9F1297F91F2012700FB21F93E
:1004500006B3237F89F2315058F1102710FB22F99F
:1004600016B3277E79F2012700FB23F92F7C81F256
:1004700006B3102710FB24F92F7971F200C016B3D0
:10048000012700FB25F92F7359F200C006B310278E
:1004900010FB26F9223040F200C016B3012700FB02
:1004A00027F9243028F64F77206816B30000F9CFDB
:1004B00010E41ABF002717C03B503195C31BD04032
:1004C00010E41ABF0881033CE9F00B34D9F0209105
:1004D00023011981110F1213EDCF093641F10D32AD
:1004E00011F0013E39F700932A013F914F911F917E
:1004F0000F912F91DF91CAB7C6FD51CFCF91CFBFDA
:10050000CF91189520912A01222379F31091280187
:10051000112311F5343012F1309328012093240176
:10052000109125013BE0311B3093250117C000914C
:10053000280101308CF40AE53091000134FD10C02F
:1005400000930001C8E1D1E00FC02795A8F45150F5
:10055000A9F4220F0000F9CF4AE503C042ED01C023
:10056000432FC4E1D0E032E017B31360C09A17BB49
:1005700008B320E413E05F93012756E008BB2795FA
:1005800020F4515021F4220FF9CF012756E000004A
:100590003B5A08BBD0F2279528F4515029F4220F7A
:1005A0000000F9CF012756E0279508BB20F45150F1
:1005B00021F4220FF9CF012756E02991332308BBFC
:1005C00021F60C7F10912901110FC651D04008BBB4
:1005D00011F01093230110E41ABF016017B31C7FC0
:1005E000402F4C7F5F9100C000C008BB17BB48BBC9
:1005F0007CCF809145018CBD809142018DBD0895D5
:10060000282F8823A1F0883008F042C082EA93E0C6
:100610009093440180934301243019F12530B8F0C0
:10062000263099F1263068F12730F9F0089583ECEF
:1006300093E0909344018093430181E080934701CC
:1006400082E58093450181E0809342010895223044
:10065000A1F0233070F4213049F780EC80934701FA
:10066000089588E180934701089583E080934701CE
:10067000089580E380934701089580E680934701C1
:1006800008958CE0809347010895209347010895D1
:1006900083EC93E0909344018093430110924201D4
:1006A00081E080934701293041F02A3050F428300E
:1006B00039F683E580934501089582E580934501ED
:1006C00008952B3029F02C3009F0BACF80934201E5
:1006D00081E580934501089526B59091470186B53F
:1006E000821B8917E0F3089584B18C6284B92A983B
:1006F0002D9896B52091470186B5891B8217E0F3A6
:100700002A9A96B586B5891B8217E0F32A988091BC
:10071000430190914401835C934019F0109246018B
:100720000895809145018CBD809142018DBD10924C
:100730004601089584B1837D84B985B1837D85B9EF
:100740001CBC0895582F2091470140E030E057FD30
:1007500016C02B98440F1C994F5F2D9A96B586B5FD
:10076000891B8217E0F32D9896B586B5891B8217F1
:10077000E0F33F5F383029F0550F57FFEACF2B9A4F
:10078000E9CF842F08958EBD0DB407FEFDCF8EB541
:1007900008950F931F930FE1E0914301F0914401FD
:1007A0008CEA0995E0914301F091440183E50995B4
:1007B000E0914301F091440180E00995182FE09108
:1007C0004301F091440180E00995133561F11CBCAF
:1007D00026B59091470186B5821B8917E0F32A9AC6
:1007E00026B586B5821B8917E0F32A9826B586B50B
:1007F000821B8917E0F3E0914301F091440183E00B
:10080000E33CF80721F0002351F00150C9CF80915B
:1008100045018CBD809142018DBD0023B1F781E07F
:100820001F910F91089580E01F910F9108959B01F2
:10083000AC0181E156954795379527958A95D1F773
:10084000809146018217D9F020934601E09143013F
:10085000F09144018DE40995E0914301F091440148
:1008600080E00995E0914301F091440180914601B7
:100870000995E0914301F091440180E009950895C4
:10088000EF92FF920F931F937B018C010E9417043C
:100890008E2D8170880F880F880FE0914301F091B1
:1008A000440180620995D801C70129E0B695A79552
:1008B000979587952A95D1F7E0914301F0914401EE
:1008C000099516950795F794E794E0914301F09107
:1008D00044018E2D0995E0914301F091440180E09F
:1008E00009951F910F91FF90EF9008950F931F931B
:1008F0008C01E0914301F091440180EA0995E09177
:100900004301F0914401812F0995E0914301F09159
:100910004401802F0995E0914301F091440180E06A
:1009200009951F910F910895FF920F931F938C01CA
:10093000F62EE0914301F091440180EC0995E0919D
:100940004301F0914401812F0995E0914301F09119
:100950004401802F0995E0914301F09144018F2DCE
:1009600009958EE10E94730580E01F910F91FF9021
:100970000895CF92DF92EF92FF920F931F936B0136
:100980007C01142F0E941704E0914301F09144016F
:100990008CE40995D701C60149E0B695A7959795CE
:1009A00087954A95D1F7E0914301F091440109956B
:1009B000D701C601B695A79597958795E091430114
:1009C000F09144010995E0914301F091440180E0E8
:1009D00009951F3FF9F016B50EE1C701B6010E9457
:1009E00040048F3F79F486B5811B8D33B0F316B583
:1009F000015099F781E01F910F91FF90EF90DF90E8
:100A0000CF90089580E01F910F91FF90EF90DF90BD
:100A1000CF9008958FE00E94730580E01F910F91A1
:100A2000FF90EF90DF90CF900895CF92DF92EF92FA
:100A3000FF920F931F936B017C01042F122F0E94D2
:100A400017048C2D8170880F880F880FE091430167
:100A5000F091440180640995D701C60169E0B6951B
:100A6000A795979587956A95D1F7E0914301F09105
:100A700044010995D701C601B695A7959795879525
:100A8000E0914301F09144010995E0914301F09117
:100A90004401802F09951123C9F00F37F9F016B5DD
:100AA0000EE1C701B6010E9440048F3779F486B584
:100AB000811B8D33B0F316B5015099F781E01F917A
:100AC0000F91FF90EF90DF90CF90089580E01F91FD
:100AD0000F91FF90EF90DF90CF9008958FE00E94EC
:100AE000730580E0F4CF382F882349F020E096B5D5
:100AF00086B5891B8C33E0F32F5F2317C0F308956D
:100B0000259A23982B9A50E217D05A95E9F7089521
:100B1000AC0188E605D0842F03D089E601D0852F6B
:100B20000FD028E030E0382780FB869506D02A9544
:100B3000D1F730FB02D000D0689423982B9A16F09E
:100B40002B98239AE0914801F09149013197F0F7F1
:100B50002D9AE3B1E3FBE0914801F091490131970F
:100B6000F0F72D98089520ECE7DF46F42A95E1F799
:100B700080E02AE1E5DF2A95E9F7DECF28E030E0E2
:100B8000DBDF869587F938272A95D1F7D5DF27F956
:100B9000322772F3D1DFD0CFDB01742FB9DF84E2CB
:100BA000BFDFE1DF8D937A95D1F70895DB01742FD4
:100BB000AFDF83EFB5DF8DE1B3DF84E6B1DF8D9189
:100BC000AFDF82E7ADDFCFDF8078D9F77A9589F79D
:100BD00008951BB815B88BEF8AB98FEF84B914B894
:100BE00093E097B98EEF88B995BD0E947C00789408
:100BF0000E948300FDCFFF920F931F93CF93DF934B
:100C0000082F792FF62E40910301413069F04430CE
:100C100059F0463009F497C01FEF812FDF91CF9133
:100C20001F910F91FF900895FF2009F4B8C0802F05
:100C3000972F9C01E90110E055C08091140190911B
:100C40001501892B09F05BC06091100170911101B1
:100C50008091120190911301488121E00E941505B5
:100C60008091040190910501019790930501809373
:100C70000401892BE1F4109203018091160181FF98
:100C80003CC08091170190E0209114013091150132
:100C90008217930791F16091100170911101809179
:100CA00012019091130148810E94B90411E08091D2
:100CB000100190911101A0911201B09113010196C0
:100CC000A11DB11D8093100190931101A0931201F9
:100CD000B093130121969E01201B2F1508F09DCF84
:100CE00040910301413009F4A8CF80911001909107
:100CF000110168810E949404B3CF11E0D8CF6091B4
:100D0000100170911101809112019091130148819D
:100D100020E00E94150580911701815080931701F2
:100D2000882309F09DCF609110017091110180918D
:100D300012019091130148810E94B904809114011D
:100D4000809317018DCF8091100190911101602F38
:100D50004F2D0E94D6058091100190911101A09114
:100D60001201B09113018F0D911DA11DB11D809332
:100D7000100190931101A0931201B093130180917F
:100D80000401909105018F199109909305018093B9
:100D90000401892B21F41092030111E03ECF10E0F1
:100DA000812FDF91CF911F910F91FF9008950F93A5
:100DB0001F93CF93DF93082F792F162F40910301B4
:100DC000842F8250823050F0453009F44AC01FEF22
:100DD000812FDF91CF911F910F910895453009F434
:100DE00040C06623B1F1802F9C01E90121C08091B0
:100DF0001001909111010E94760488838091100166
:100E000090911101A0911201B09113010196A11DC1
:100E1000B11D8093100190931101A0931201B09322
:100E2000130121969E01201B211780F4409103019C
:100E30004230E9F660911001709111018091120128
:100E4000909113010E9440048883D8CF183008F095
:100E5000BFCF10920301812FDF91CF911F910F918E
:100E600008958091100190911101602F412F0E94EF
:100E7000CC058091100190911101A0911201B091C7
:100E80001301810F911DA11DB11D8093100190933D
:100E90001101A0931201B09313019ACF0F931F93E6
:100EA000CF93DF938C01DC0111968C91813009F492
:100EB0004EC0823009F4EAC0833009F457C0843050
:100EC00009F4B8C0873009F489C0853009F45EC1DF
:100ED000863009F414C1883009F4DFC0893009F480
:100EE0005DC18A3009F46EC18B3009F4A1C18C3028
:100EF00009F4BFC18D3009F4D8C18E3009F4DDC1C9
:100F00008F3009F06AC1F801938180E0228130E0DE
:100F1000822B932BAA2797FDA095BA2F80931001BF
:100F200090931101A0931201B0931301978180E077
:100F3000268130E0822B932B90930501809304014E
:100F400085E0809303018FEFC8E0D1E03AC0329B87
:100F500041C0809106010E94000310920701419850
:100F60000E94740380E0C8E0D1E02BC0E09143010F
:100F7000F0914401D80112968C910995C8E0D1E016
:100F800080930801E0914301F0914401D801139648
:100F90008C91099580930901E0914301F0914401FE
:100FA000D80114968C91099580930A01E091430130
:100FB000F0914401D80115968C91099580930B010D
:100FC00084E0D0932701C0932601DF91CF911F9138
:100FD0000F91089585E00E940003BFCF8091070123
:100FE000882399F4F801938180E0228130E0822BFC
:100FF000932BAA2797FDA095BA2F80931001909369
:101000001101A0931201B0931301D80117969C917E
:10101000179780E016962C9130E0822B932B9093BB
:1010200005018093040183E0809303018FEFC8E002
:10103000D1E0C7CF80910701882399F4F80193810B
:1010400080E0228130E0822B932BAA2797FDA09588
:10105000BA2F8093100190931101A0931201B093C5
:101060001301D80117969C91179780E016962C9142
:1010700030E0822B932B909305018093040182E052
:10108000809303018FEFC8E0D1E09BCF0E949A03C9
:10109000419A80E0C8E0D1E094CF80910701882395
:1010A000B1F4D80113969C91139780E012962C917D
:1010B00030E0822B932BAA2797FDA095BA2F80931F
:1010C000100190931101A0931201B093130110929B
:1010D00015011092140110921601F801978180E019
:1010E000268130E0822B932B90930501809304019D
:1010F00084E0809303018FEFC8E0D1E062CF80915C
:101100000701882399F4F801938180E0228130E07F
:10111000822B932BAA2797FDA095BA2F80931001BD
:1011200090931101A0931201B0931301D80114966A
:101130008C91149715969C91292F2F70209316014E
:10114000492F50E0407F507042955295507F542770
:10115000407F5427480F511D5093150140931401AF
:1011600020FF02C040931701F801978180E026819B
:1011700030E0822B932B909305018093040181E052
:10118000809303018FEFC8E0D1E01BCF0E94C90319
:10119000C8E0D1E08093080181E013CF81E0809323
:1011A0000701F80182819381A481B58180931001A8
:1011B00090931101A0931201B093130180E0C8E055
:1011C000D1E0FFCED80112968C9180930601C8E041
:1011D000D1E01092080181E0F4CE803109F043C0E3
:1011E000D80113969C91139780E012962C9130E0D1
:1011F000822B932BAA2797FDA095BA2F80931001DD
:1012000090931101A0931201B0931301F8019781FB
:1012100080E0268130E0822B932B90930501809310
:10122000040186E0809303018FEFC8E0D1E0C9CECE
:10123000F801938180E0228130E0822B932B909300
:101240004901809348012A9A229A83E00E947305FB
:101250002A98419880E10E9473050E94800580E0F1
:10126000C8E0D1E0AECE8F3789F180E0C8E0D1E0B0
:10127000A8CE80EC0E94900580E00E9490058AE054
:101280000E9473052A9A85E00E9473052A9885E0DA
:101290000E94730584B1837D84B985B1837D85B94E
:1012A000419A80E0C8E0D1E08CCE0E94B305C8E04E
:1012B000D1E08093080181E084CED80112968C9110
:1012C0000E94900580E0C8E0D1E07BCEC8E0D1E08C
:1012D00081E0809308011092090110920A01109296
:0A12E0000B0184E06ECEF894FFCFFE
:0212EA005AFFA9
:00000001FF
